:1000000000308A00402F0000831A0A28A500030E42
:10001000A6000F288312A500030EA600A6140A0846
:10002000AD008A018313A50E0408A7002008A800CC
:100030002108A9002208AA002308AB002408AC006C
:1000400083128B1E25280B19282D270884002808C9
:10005000A0002908A1002A08A2002B08A3002C0850
:10006000A4002D088A00260E83008312250EA618F0
:10007000831609000A108A100A1182077434653445
:100080006D3470340934253433342E3431346634CD
:1000900046340934253433342E3431346634433411
:1000A0000D340A3400340A108A100A1182074E34C3
:1000B00065347734203473346534633473343A34BC
:1000C000203400340A108A100A1182070D340A34D1
:1000D00053346534633473343A342034253464340F
:1000E0000D340A3400348E30A0004908A1004808BD
:1000F000A200A301A108031D87282208A100A201D4
:100100000830A002A108031D8728A0018F28031032
:10011000A11B8E28A20DA10DA0038728A11300000A
:1001200000345C0803190129E4006008031901295F
:10013000E4070318A2287F30E402031C01290319F5
:100140000129A6288130E407031801296408A000CA
:10015000A101A201A3015D08E800E8175E08E7001D
:100160005F08E6001830E400E501661CCF2863084C
:10017000A307031CC128A20A031DC128A10A031951
:10018000E5176208A207031CC828A10A0319E5178E
:100190006108DE00DE175E08A1070318E517E50D0C
:1001A000A10CA20CA30CE80CE70CE60C0310E40B6A
:1001B000B4280130A00703180129A11BE628E80D87
:1001C000A30DA20DA10DA00303190129E81FF72813
:1001D000A30A031DF728A20A031DF728A10A031D7D
:1001E000F728A10CA20CA30CA00A031901295D0891
:1001F000E5006108E506E51FFF28A1170529A11301
:100200000529A001A101A201A301000000344908B1
:10021000D0004D08D006D01F122903110310C91BAE
:10022000031445294908D0004C08D1004808D102E0
:1002300003192029D01F45290308013A83004529C5
:100240004D08D1004908D10203192C29D01F452996
:100250000308013A830045294E08D1004A08D1021B
:1002600003193829D01F45290308013A830045297D
:100270004F08D1004B08D10203194429D01F45294A
:100280000308013A8300452903105A2D83160511EE
:1002900083120511A630A000A00B4C290000831684
:1002A0000515A6308312A000A00B54290000831668
:1002B000051583120034CE014E08073C031C7D292E
:1002C0008316051183120511000000000310CD0CE8
:1002D00003186C2905116D290515831605111330B6
:1002E0008312A000A00B72290000000083160515E0
:1002F000000000008312CE0A5C290034CD014D08B5
:10030000073C031CA2298316051183120511000066
:1003100000008316051502308312A000A00B8E2961
:1003200000008316051583120519982903109929D1
:100330000314CE0C2730A000A00B9C290000000065
:10034000CD0A7F294E08A10000348E30A0004E084F
:10035000A1004D08A200A301CE1FB329A109A20943
:10036000A20A0319A10AA108031DC0292208A1009D
:10037000A2010830A002A108031DC029A001C929BB
:100380000310A11BC729A20DA10DA003C029CE1FD8
:10039000A1130000822D51080319902ADD00550891
:1003A0000319902ADD02031CDA297F30DD070318C8
:1003B000902AE0298130DD02031C902A0319902A3B
:1003C0005D08A000A101A201A301DC015208DB002D
:1003D000DB175308DA005408D9001930DD0058083B
:1003E000D9020318032A0130DA020318032ADB02B8
:1003F0000318032ADC020318032ADC0ADB0ADA0AE0
:100400005808D907352A5708DA0203181E2A01307E
:10041000DB0203181E2ADC0203181E2ADC0ADB0A90
:100420005708DA075808D907031C352ADA0A031DCA
:10043000352ADB0A031D352ADC0A352A560880389E
:10044000DB020318342A0130DC020318342ADC0AE8
:1004500056088038DB075708DA07031C122ADB0A24
:10046000031D122ADC0A122A2314DD0B382A432A20
:100470000310D90DDA0DDB0DDC0D0310A30DA20D59
:10048000A10DDE0DEF295E1C4B2A0310A10CA20C5E
:10049000A30CDE0C4E2AA0030319902ADE1B772A38
:1004A0000310D90DDA0DDB0DDC0D5808D902031845
:1004B000632A0130DA020318632ADB020318632A75
:1004C000DC02031C862A5708DA0203186E2A013060
:1004D000DB0203186E2ADC02031C862A56088038C9
:1004E000DB020318772A0130DC02031C862AA30AE8
:1004F000031D862AA20A031D862AA10A031D862A35
:10050000A00A0319902AA10CA20CA30C5208DD002A
:100510005608DD06DD1F8E2AA117942AA113942AFE
:10052000A001A101A201A301000000344D3084000C
:1005300000080319AA2A0130A100A001A00B9E2ADD
:10054000A10B9D2A4A30A000A00BA42A00000000A5
:10055000800B9B2AA22D80308318D106D601D701AB
:100560004D08D5005108D5064C080319982BD40026
:10057000A00050080319A12BD40203193E2B031C21
:10058000FD2A5108DA00DA175208D9005308D800BA
:10059000D7010310DA0CD90CD80CD70CD40BC82A0D
:1005A000D51FD52A5614B52B5610541056164F3059
:1005B0008400CA2B5612D51BE72A541CF22ADA0CE7
:1005C000D90CD80CD70CA00A0319B02BF22ADA1BCD
:1005D000F52A0310D70DD80DD90DDA0DA003031994
:1005E000B02BE72A56175D2B56134D08D500CD1FAB
:1005F000FB2ADA17A92BDA13A92B5008D400A00084
:100600004C08D4024D08DA00DA174E08D9004F081A
:10061000D800D7010310DA0CD90CD80CD70CD40BA6
:10062000092BD51F162BD614B52BD6105410D61661
:1006300053308400CA2BD612D51B282B541C332BC5
:10064000DA0CD90CD80CD70CA00A0319B02B332B19
:10065000DA1B362B0310D70DD80DD90DDA0DA003F8
:100660000319B02B282BD6175D2BD6135108D500B4
:10067000D11F3C2BDA17A92BDA13A92B5108DA006A
:10068000DA175208D9005308D800D51F4B2BDA13BC
:100690005615B52B5611D70154104F308400CA2B74
:1006A000D51B732B4D08D500541C5D2BDA0CD90CCF
:1006B000D80CD70CA00A0319B02BD71F6E2BD80A61
:1006C000031D6E2BD90A031D6E2BDA0A031D6E2B38
:1006D000DA0CD90CD80CA00A0319B02B561BF42A3B
:1006E000D61B352B922B8030DA06DA1F7B2BB52BED
:1006F0005108D500882B4D08D500DA08031D882B3A
:10070000D908031D882BD808031D882BA001A92B0D
:10071000DA1B922B0310D70DD80DD90DDA0DA00BD3
:10072000882BB02BD51F962BDA17A92BDA13A92B00
:100730005008A0005108DA005208D9005308D80028
:10074000A92B4C08A0004D08DA004E08D9004F082C
:10075000D8005A08A1005908A2005808A300E82BA5
:10076000A001A101A201A301E82BD701D809D90951
:10077000DA09D709D70A031DC32BD80A031DC32BD7
:10078000D90A0319DA0A5618D42AD618152B56197D
:100790004A2B782B0008D807031CD42BD90A031D39
:1007A000D42BDA0A0319541484030008D907031C54
:1007B000DC2BDA0A0319541484030008801F803AE2
:1007C000DA0703185414561ADA2AD61A1B2B502BA0
:1007D0000000EE2D83160510831205100830A100CD
:1007E000000000000000A117042CA113DC0C03186A
:1007F0000514031C05102117042C2113A10BF62B43
:1008000000000000000005141C308400840B062C3E
:10081000A11BF52B211BFD2B00345C08B63CDC0032
:10082000A3015D08E000DD170310DD0CDE0CDF0C1A
:10083000A30CA20CA10CA00CDC0B142CE01F2B2C85
:10084000A009A109A209A309A00A0319A10A031971
:10085000A20A0319A30A962CA001A101A201A301D7
:10086000E401E501E601E701630862046104600454
:1008700003196A2C2030E8000310DC0DDD0DDE0DBD
:10088000DF0DE40DE50DE60DE70D63086702031DBE
:10089000532C62086602031D532C61086502031D78
:1008A000532C60086402031C642C6008E402610895
:1008B000031C610FE5026208031C620FE602630875
:1008C000031C630FE7020314A00DA10DA20DA30DDD
:1008D000E80B3C2C00006430840000340408D6008F
:1008E0005508D70003198D2C5408DF005308DE008B
:1008F0005208DD005108DC00E301E2012030E10094
:100900008230E00091202308D4002208D30021087F
:10091000D2002008D100D70B742C5408DF005308F4
:10092000DE005208DD005108DC000D2C2308D40045
:100930002208D3002108D2002008D100D41FAD2CFA
:10094000D603D616D109D209D309D409D10A03197D
:10095000D20A0319D30A0319D40A3B30DB009A30B8
:10096000DA00CA30D900D8010A30D7005508031977
:10097000D60A5408DF005308DE005208DD00510893
:10098000DC005B08E3005A08E2005908E10058085F
:10099000E0002C240008D100840A0008D200840A58
:1009A0000008D300840A0008D400FD308407A008A2
:1009B000031DEB2C550A57020319EB2C560803199B
:1009C000ED2C0F3957020319E72C03180F2D561B76
:1009D000ED2C20300B2D2030D60555085702031D75
:1009E000FB2C2008D6002E30DC00EA235608A0009D
:1009F0002030D60500303030D61E0B2DD6125508CB
:100A0000031DD6032008D6002D30DC00EA2356084B
:100A1000A000D6013030A0072008DC00EA235B08E4
:100A2000DF005A08DE005908DD005808DC00E30149
:100A3000E201E1010A30E0002C242308DB00220857
:100A4000DA002108D9002008D800D70BB92C0034CF
:100A5000C9013108C80073202308DF002208DE0026
:100A60002108DD002008DC000A30E300D730E20076
:100A70002330E1007B30E00091202008C4002108F1
:100A8000C5002208C6002308C700C9013608C800EF
:100A900073202308CB002208CA002108C9002008BF
:100AA000C8004708CF004608CE004508CD004408DE
:100AB000CC000729031C2A2EB101C4014621CC30E9
:100AC000CD005B214430CD005B21C408031D6C2D9B
:100AD0007E212108C400652D4621CC30CD005B214C
:100AE000BE30CD005B217E212108C5007E2121087A
:100AF000C6004608C8004508C7004808CE00470899
:100B0000CD00A5292008CD002108CE002208CF0065
:100B10002308D000D4002208D3002108D2002008E6
:100B2000D100D801D701D6018330D500CB212308CD
:100B3000CC002208CB002108CA002008C900C83018
:100B4000CD00962A4908A0004A08A1004B08A2003F
:100B50004C08A3002308B5002208B4002108B30004
:100B60002008B2003508DF003408DE003308DD005D
:100B70003208DC00E301E2011030E1008230E000E5
:100B800091202008C4002108C5002208C6002308BF
:100B9000C700D4002208D3002108D2002008D100C9
:100BA000D801D7012030D6008130D500CB212008D4
:100BB000C8002108C9002208CA002308CB008310FE
:100BC0002308CF002208CE002108CD002008CC0049
:100BD000D301D201D1018430D000AB2A2008CC004F
:100BE0002108CD002208CE002308CF00D0015008F4
:100BF0003A20D00AA000DC00EA2305305002031D91
:100C0000F72D023084004F08D4004E08D3004D0861
:100C1000D2004C08D1000130D5006E244630DC00F3
:100C2000EA230930DC00EA23023084003508D400CE
:100C30003408D3003308D2003208D1000130D50087
:100C40006E244330DC00EA230D30DC00EA230A3056
:100C5000DC00EA23B10A0B118A1125280308183990
:100C6000A00083160E0803398312200483160E1485
:100C70008E14183A8312031D3E2E3F2E3F2E1F1353
:100C800083161F109F101F119F1183121F10003019
:100C9000A1005E2F0830A000831685148312851CE6
:100CA000532E83164E2EBD01A017642EA013642E62
:100CB000031085180314BD0C2017642E2013A00BFD
:100CC000582E3D08A100702E1C30A01B0730A1003B
:100CD000A10B682E0000A01B562E201B5E2E582E46
:100CE00000344A262108BC00AE018B1BAE178B13C3
:100CF0003C08DC00EA23AE1B8B173C08393C031C84
:100D0000862E30303C02A100962E962E3C08603C88
:100D10000318912E3C087A3C031C912E3C08DF39C5
:100D2000922E3C08BF3E0A3EA100962E003471264A
:100D30002108BB0071262108BA003A08DD3C031DDA
:100D4000A52E3B08A100AD2EAD2E3B0EA000F0302D
:100D5000A00520083A07A100AD2EA42F4208A1014A
:100D600041020318B62E4108A000C22EA00108308F
:100D7000C300C10DA00D420820020318A000A10D60
:100D8000C30BB92E003420303C1E3030BD003B0870
:100D9000A000BB1FD22EA009A00A2008BB002D3046
:100DA000BD00BC173B08C1006430C200AE2620085D
:100DB000BB0030302107BE003B08C1000A30C20032
:100DC000AE2630302007C00030302107BF003D087C
:100DD000A000BC1DED2EBC1F3C113C1AFA2EBC1FFE
:100DE000152F3C19152F2008BE00BC18152F200800
:100DF000BF00152F30303E02031D152F2008BE0006
:100E00002030BD00BC1D082F3C11BC14BC1FBC1001
:100E100030303F02031D152F2008BF002030BE00D8
:100E2000BC1D082FBC10BC1F3C103C1D202FAE0168
:100E30008B1BAE178B133D08DC00EA23AE1B8B1710
:100E4000BC1C2B2FAE018B1BAE178B133E08DC0096
:100E5000EA23AE1B8B173C1C362FAE018B1BAE1743
:100E60008B133F08DC00EA23AE1B8B17AE018B1BF4
:100E7000AE178B134008DC00EA23AE1B8B17BD2F87
:100E800084011F3083051F1383161F109F101F112D
:100E90009F11073083129900613083168F000F086D
:100EA000051083120514AF01B101B201B301B40101
:100EB000B5010330B600B701B8012E2E8316051216
:100EC000831205128B16C0308B0483160108C039BB
:100ED0000738810083128101AE018B1BAE178B1383
:100EE0003E30DC00EA23AE1B8B17AE018B1BAE1726
:100EF0008B132030DC00EA23AE1B8B174A26210817
:100F0000B9008B123908703A03198D2F5B3A031917
:100F1000D42F063A0319D92FDE2F83160512831218
:100F20000516BA013A085320BA0AA000AE018B1B7D
:100F3000AE178B132008DC00EA23AE1B8B170A3098
:100F40003A02031D922F972E2108B600BA013A08E3
:100F50006220BA0AA000AE018B1BAE178B132008CB
:100F6000DC00EA23AE1B8B1708303A02031DA72FC3
:100F70003608BB001F30BC00C32EAE018B1BAE1762
:100F80008B130D30DC00EA23AE1B8B17AE018B1BDD
:100F9000AE178B130A30DC00EA23AE1B8B178316C7
:100FA000051283120512FA2F8316051283120516F5
:100FB000FA2F8316051283120512FA2FAE018B1B2E
:100FC000AE178B133908DC00EA23AE1B8B17AE017A
:100FD0008B1BAE178B130D30DC00EA23AE1B8B1777
:100FE000AE018B1BAE178B130A30DC00EA23AE1B5D
:0A0FF0008B17FA2F8B166C2F63008D
:02400E00C43CB0
:00000001FF
